:06000000020F5D02006B1F
:03000B0002006B85
:0300130002006B7D
:03001B0002006B75
:0300230002006B6D
:03002B0002006B65
:0300330002006B5D
:03003B0002006B55
:0300430002006B4D
:03004B0002006B45
:0300530002006B3D
:03005B0002006B35
:0300630002006B2D
:01006B003262
:1000800002006B0002006B0002006B0002006B00BC
:1000900002006B0002006B0002006B0002006B00AC
:1000A00002006B0002006B0002006B0002006B009C
:0800B00002006B0002006B006E
:1001000002006B0002006B0002006B0002006B003B
:1001100002006B0002006B0002006B0002006B002B
:1001200002006B0002006B0002006B0002006B001B
:1001300002006B0002006B0002006B0002006B000B
:1001400002006B0002006B0002006B0002006B00FB
:1001500002006B0002006B0002006B0002006B00EB
:1001600002006B0002006B0002006B0002006B00DB
:1001700002006B0002006B0002006B0002006B00CB
:030F6300020F6614
:030F7900020180F2
:100180001205CF80FEC200E4F508F509F50AD20198
:10019000750B00750C001207CC1207C975CB63757F
:1001A000CAC0758E0075C804D2AFD2B0D2B190E685
:1001B0000B7403F00090E6047480F00090E6047481
:1001C00002F00090E6047404F00090E6047406F077
:1001D0000090E6047408F00090E604E4F00090E675
:1001E0001074A0F00090E61174A0F00090E618E4FE
:1001F000F00090E61274A2F00090E619E4F000908E
:10020000E61374A0F00090E60BE4F00090E614749E
:10021000A2F00090E61AE4F00090E61A7411F000E3
:1002200090E61574E0F00090E61BE4F00090E61B09
:100230007409F00090E626E4F00090E6277440F0A0
:100240000090E6917480F00090E6957480F0009044
:10025000E6917480F00090E6957480F00043A080F1
:1002600090E6FBE0FA54FDF090E601E0FA54F7F076
:1002700022AA82850C827583E0EAF0050C0509E468
:10028000B50902050A22200001221207C890E6A241
:10029000E0FA30E10302031FE509450A60697AC00C
:1002A0007BE78B9D7AC07BE77B008A9E90E67C741F
:1002B00031F07460F0C3743E9509E4950A50107AE9
:1002C0003EE50924C2F509E50A34FFF50A8007AACC
:1002D00009E4F509F50A8A037C007DE08D9A850B17
:1002E0009B8A041AEC601190E67BE0FC90E67CF0BF
:1002F0007C007DE08D9A80E9859B0B0090E68F74F1
:10030000022BF0D2CF801830CF1590E7C07431F0B7
:1003100090E7C17460F00090E68F7402F0C2CFE500
:10032000AA30E00122C3E50994C1E50A9400400126
:100330002290E690E0FA8A037A0090E691E0FC7D54
:1003400000EA4CF50DEB4DF50E7C007DF08D9A7CAE
:10035000007DF07D008C9B7C007D00C3EC950DED55
:10036000950E4003020457E5087003020407E50DEB
:10037000C39CFEE50E9DFFA8087900C3E89EE99F97
:100380005004880689078E00E508C398F508EE2C0E
:10039000FCEF3DFD30012D8E008F0188028903188E
:1003A000B8FF0119EA4B60B390E67BE0FAF582C032
:1003B00004C005C000C001120820D001D000D00543
:1003C000D00480D78E028F038A068B071ABAFF01EA
:1003D0001BEE4F700302035B90E67BE0FEF582C0EC
:1003E00002C003C004C00512085DD005D004D003CC
:1003F000D002C002C003C004C005120271D005D0F3
:1004000004D003D00280C190E67BE0FA30E6047BA2
:100410000080027B01EB24FF9201EA30E707743F82
:100420005AF508802A30010F8A82C004C0051207DD
:10043000E2D005D00480188A82C004C005120812D8
:10044000D005D004C004C005120271D005D0040C40
:10045000BC00010D02035B0090E6917480F02290D5
:10046000E6B8E0FA20E70C90E6B9E07002D2007539
:1004700082012290E6B9E0FABA9002801ABA91029B
:10048000805ABA9203020514BA930302052EBA9455
:100490000302055E02059790E6BCE025E0547FFA72
:1004A0002400F582E43418F583E0FB90E740F07413
:1004B000012A2400F582E43418F583E0FA90E7413C
:1004C000F090E6BEE0FABA0200500790E6BEE0FA0D
:1004D00080027A0290E68BEAF00205C090E6BCE06A
:1004E000701390E6FBE0FA54FDF090E7407402F0E0
:1004F0001208F2801190E6FBE0FA4402F090E74027
:100500007401F01208F290E68AE4F090E68B740130
:10051000F00205C090E6BCE0700543A08080035364
:10052000A07F90E68AE4F090E68BF00205C090E6AA
:10053000BCE0700F90E601E0FA54F7F090E740E479
:10054000F0800E90E601E0FA4408F090E740740174
:10055000F090E68AE4F090E68B7401F080627A0015
:100560007B00EA247CFCEB340FFD7E808C828D8343
:100570008EF0120F41FC6013EA2440F582EB34E761
:10058000F583ECF00ABA00DA0B80D790E68AE4F043
:1005900090E68BEAF0802990E7407436F090E741CE
:1005A0007483F090E68AE4F090E6BEE0FABA0200C6
:1005B000500790E6BEE0FA80027A0290E68BEAF0FD
:1005C00075820122300203120A8D12028680F5C262
:1005D000AF12018512062C120E721209F7D2AF1259
:0505E00008F20205C451
:060F7C00342E322E30007D
:10E100001201100100000040C016AD06040001021B
:10E1100003010A061001FFFFFF400100090237005A
:10E1200002010080FA0904000002FFFFFF02070558
:10E1300081024000000705020240000009040100BE
:10E1400002FFFFFF02070506020002000705880222
:03E15000000200CA
:10E154001201100100000040C016AD0604000102C7
:10E1640003010A061001FFFFFF4001000902370006
:10E1740002010080FA0904000002FFFFFF02070504
:10E18400810240000007050202400000090401006A
:10E1940002FFFFFF02070506024000000705880290
:10E1A40040000004B0E1B6E1C0E1D8E1060300009C
:10E1B40009040A034500500046004C0018035500AA
:10E1C400530042002D004A005400410047002D0036
:10E1D40049004600120330003000300030003000A7
:06E1E400300030003000A5
:1005E500AA82E50F54FEFBB50F02802A8A048C050A
:1005F500E4FC6210ED6211EB2400F582E43418F599
:1006050083E0FB7C006210EC6211E51033C5113309
:10061500C51192E0F510AB0F050FEB2400F582E450
:100625003418F583EAF022750F007510AA7511AA22
:100635007582001205E57582001205E57A00C3EAA8
:10064500648094865018EA2408F582E434E1F58341
:10065500E0FBF582C0021205E5D0020A80E07A00CF
:10066500C3EA648094825018EA2423F582E434E1D5
:10067500F583E0FBF582C0021205E5D0020A80E0B1
:1006850075821C1205E57582001205E57A00C3EA3C
:10069500648094825018EA2402F582E434E1F583FB
:1006A500E0FBF582C0021205E5D0020A80E07486FF
:1006B500250FFAF582C0021205E5D00290E1B6E0F9
:1006C500FBF582C0021205E5D00290E1B6E0FB2AF7
:1006D500FAF582C0021205E5D00290E1C0E0FBF513
:1006E50082C0021205E5D00290E1C0E0FB2AFAF5CE
:1006F500821205E590E1D8E0FAF5821205E57A0067
:1007050090E1B6E0FBC3EA64808BF063F08095F07E
:100715005018EA24B6F582E434E1F583E0FBF5826E
:10072500C0021205E5D0020A80D67A0090E1C0E049
:10073500FBC3EA64808BF063F08095F05018EA24DF
:10074500C0F582E434E1F583E0FBF582C0021205D1
:10075500E5D0020A80D67A0090E1D8E0FBC3EA64CE
:10076500808BF063F08095F05018EA24D8F582E488
:1007750034E1F583E0FBF582C0021205E5D0020AFB
:1007850080D67A00C3EA648094845018EA240EF572
:1007950082E434E1F583E0FBF582C0021205E5D081
:1007A500020A80E07482250F40087582001205E573
:1007B50080F2AA107B0090187EEAF0AA1190187FAB
:1007C500EAF0222222222290E6007412F090E6013D
:1007D5007403F0AAB574FD5A440DF5B522E582FA05
:1007E50030E0047B0180027B00EB24FF92B3EA300A
:1007F500E1047B0180027B00EB24FF92B2EA30E446
:10080500047A0180027A00EA24FF92B0221207E2FC
:10081500E4A2B133FA74024AF58222E5821392B05A
:10082500D2B313C2B392B0D2B313C2B392B0D2B3A0
:1008350013C2B392B0D2B313C2B392B0D2B313C240
:10084500B392B0D2B313C2B392B0D2B313C2B392C0
:10085500B0D2B300C2B32222E582A2B11392B0D2C4
:10086500B3C2B3A2B11392B0D2B3C2B3A2B11392C1
:10087500B0D2B3C2B3A2B11392B0D2B3C2B3A2B1D4
:100885001392B0D2B3C2B3A2B11392B0D2B3C2B372
:10089500A2B11392B0D2B3C2B3A2B11392B0D2B384
:1008A500C2B3F58222227880E84400600C79019079
:1008B5001800E4F0A3D8FCD9FAD083D082F6D8FD8D
:1008C500C082C0837582002290E6A0E0FA4401F060
:1008D50022AA8274805AFBC423541FFB740F5A90BA
:1008E500E6834BF090E683E0FA4420F02290E68020
:1008F500E0FA440AF09000FA120F2E90E65D74FFBC
:10090500F090E65F74FFF05391EF90E680E0FA54C3
:03091500F7F022D6
:060F7300E478FFF6D8FD52
:060F5D007512007513007F
:1009180090E680E0FA30E7267514007515E1751643
:10092800127517E175181C7519E1751A70751BE1B8
:1009380090E6267402F00090E627E4F00022751491
:10094800547515E17516667517E17518707519E116
:10095800751A1C751BE190E626E4F00090E62774F2
:1009680040F000225391EF75A100D20232C0E0C0DE
:10097800F0C082C083C002C003C004C005C006C066
:1009880007C000C001C0D075D0005391EF75A10019
:10099800120918D0D0D001D000D007D006D005D089
:1009A80004D003D002D083D082D0F0D0E032C0E0AF
:1009B800C0F0C082C083C002C003C004C005C00626
:1009C800C007C000C001C0D075D0005391EF75A119
:1009D80000120918D0D0D001D000D007D006D00519
:1009E800D004D003D002D083D082D0F0D0E032122D
:1009F8000918751C6C751D09758200120DC3751CCC
:100A080075751D09758210120DC3751CB6751D0903
:100A1800758214120DC390E65C7431F022E582549D
:100A28007FFA24F7500475820022BA010475820106
:100A380022530201E4BA000104F58222AA82BA0113
:100A48000C90E6A1E0FB7C008B828C8322BA810C9F
:100A580090E6A2E0FB7C008B828C832253027FEA23
:100A6800700C90E6A0E0FB7C008B828C832290E6E1
:100A7800A3E0FB7C00EAC313FA7D00EA2BFBED3C04
:100A88008B82F58322C20290E6B8E0FA530260BA7C
:100A980000028028BA2002800DBA4002800EBA6097
:100AA800028003020D571208CD020D5712045FE5AC
:100AB800826003020D571208CD020D5790E6B8E088
:100AC800FA530280BA80028003020C5090E6B9E023
:100AD800FABA0003020BC7BA06028035BA080280C8
:100AE80008BA0A028017020C4A90E740E512F09013
:100AF800E68AE4F090E68B7401F0020D5790E74027
:100B0800E513F090E68AE4F090E68B7401F0020DAC
:100B18005790E6BBE0FABA01028017BA02028038A1
:100B2800BA03028059BA0602801BBA0702803C0247
:100B38000BC1AA14AB1590E6B3EBF07B0090E6B4BA
:100B4800EAF0020D57AA16AB1790E6B3EBF07B005C
:100B580090E6B4EAF0020D57AA18AB1990E6B3EB89
:100B6800F07B0090E6B4EAF0020D57AA1AAB1B908E
:100B7800E6B3EBF07B0090E6B4EAF0020D5790E69E
:100B8800BAE0FA90E1A7E0FBC3EA9B40061208CD61
:100B9800020D5790E6BAE0FA75F002A424A8F5828F
:100BA80074E135F0F583E0FAA3E0FB90E6B3F07B5F
:100BB8000090E6B4EAF0020D571208CD020D5790E6
:100BC800E6B8E0FA53021FBA0002800ABA010280AE
:100BD8001BBA0268802C90E740E4F090E741F0905F
:100BE800E68AF090E68B7402F0020D5790E740E435
:100BF800F090E741F090E68AF090E68B7402F002FC
:100C08000D5790E6BCE0FAF582120A25E5826026C7
:100C180090E6BCE0FAF582120A44E0FA5302019029
:100C2800E740EAF090E741E4F090E68AF090E68B3E
:100C38007402F0020D571208CD020D571208CD02AA
:100C48000D571208CD020D5790E6B9E0FA24F4507A
:100C580003020D54EA2A2A900C6373020D54020C05
:100C68009C020D1A020CFB020D54020D54020D5485
:100C7800020D54020D54020C87020D54020C9353BA
:100C8800B1BF90E6BAE0F512020D5790E6BAE0F56A
:100C980013020D5790E6B8E0FA53021FBA0002801B
:100CA80005BA024A800A90E6BAE01208CD020D574A
:100CB80090E6BAE0703390E6BCE0FAF582120A25B5
:100CC800E582602590E6BCE0FAF582120A44AA8221
:100CD800AB83E0FC5304FE8A828B83ECF090E6BC85
:100CE800E0FAF5821208D680661208CD80611208F3
:100CF800CD805C90E6B8E0FA53021FBA005190E646
:100D0800BAE0FABA01028005BA020280421208CD9E
:100D1800803D90E6BAE0FA702E90E6BCE0FAF582E3
:100D2800120A25E582601B90E6BCE0FAF582120AF9
:100D380044AA82AB83E0FC4304018A828B83ECF0F3
:100D4800800D1208CD80081208CD80031208CD90BE
:100D5800E6A0E0FA4480F022AA82BA03004005EA3D
:100D6800249C500122740F5AFBBB03028007740FA6
:100D78005AFBBB0B45A2AF9203C2AFEA2400F5822F
:100D8800E43400F5837402F07B0074012AFCE43B30
:100D9800FDEC2400F582ED3400F583E51DFCF074CC
:100DA800022AFAE43BFBEA2400F582EB3400F583DF
:100DB800AA1C7B00EAF0A20392AF22E582FA248300
:100DC80050012274035AFB600122A2AF9204C2AF01
:100DD800EA2400F582E43401F5837402F07B0074A0
:100DE800012AFCE43BFDEC2400F582ED3401F58397
:100DF800E51DFCF074022AFAE43BFBEA2400F582C4
:100E0800EB3401F583AA1C7B00EAF0A20492AF221E
:100E1800AA82BA80004005EA244B50012274035A82
:100E2800FB600122A2AF9205C2AFEA2480F582E4FA
:100E38003400F5837402F07B0074012AFCE43BFD66
:100E4800EC2480F582ED3400F583E51DFCF0740296
:100E58002AFAE43BFBEA2480F582EB3400F583AA06
:100E68001C7B00EAF0A20592AF22C2E8C2EA751C18
:100E780000751D01758243120D60751C80751D007B
:100E8800758253120D600090E650E4F00090E6522F
:100E9800E4F00090E654E4F00090E656E4F00090A8
:100EA800E65174FFF00090E65374FFF00090E655A9
:100EB80074FFF00090E65774FFF00090E658E4F0F5
:100EC80090E65974FFF090E65AE4F090E65B74FF00
:100ED800F090E65CE4F090E65D74FFF090E65EE486
:100EE800F090E65F74FFF00090E660E4F00090E6B2
:100EF8006174FFF090E662E4F090E66374FFF090AE
:100F0800E665E4F090E668740BF05391AFD2E8D24E
:100F1800EA2222AA82120F1ADAFB2290FB50A3E5DA
:100F280082458370F922AA82AB83120F231ABAFF73
:090F3800011BBA00F5BB00F22216
:0D0F66007581201208ABE582600302018056
:100F410020F71430F6148883A88220F507E6A883D9
:0C0F510075830022E280F7E49322E02286
:00000001FF
